:0400000007EF00F016
:1000080006823DED00F049EF00F0000E926E000E02
:10001800946E0F0EC16EF28EF288F28C000E826E14
:10002800000E026E640E016E25EC00F08268000E70
:10003800026E640E016E25EC00F012EF00F007EF7F
:1000480000F0000E056E000E046E2DEF00F0044A5D
:10005800052A0450015C0250800A036E0550800A8C
:100068000358D8B03AEF00F03CEF00F02BEF00F067
:1000780012000600F2A243EF00F045EF00F046EF51
:1000880000F0801EF292069211000690069200017E
:0400980009EF00F07C
:020000040020DA
:08000000FFFFFFFFFFFFFFFF00
:020000040030CA
:0E000000FF071F1FFF8285FF0FC00FE00F409C
:00000001FF
